:020000040000FA
:040000006C303A28FE
:040004000034003490
:08000800A000030EA100831209
:100010008B1C32288B1032181428B21C3228643002
:10002000010203183128182800001628172818285C
:1000300019281A281B281C281D281E281F283210A2
:10004000B214A810031005190314AA0DA90DA80DC8
:10005000B10B322832152A08AF002908AE00280853
:10006000AD00B21081010B11210E8300A00E200EF5
:02007000090085
:0C007400203084008001840A80300402E7
:10008000031C3C281230B1009F2183160C308505DB
:1000900087018312850187010730990000309A009B
:1000A000103083168E008312603083168F00831207
:1000B00000308316910000008312C830831681003F
:1000C000831231309000003083168C008312103080
:1000D0008B00BD1B7128851971286400851D6D2852
:1000E000F421EC2181018E018F010B118B100B107B
:1000F0008C018B17892032199F20B40B872803109D
:1001000085190314BA0DF0303A0203191821192287
:100110007A286400321808000B1D08000B11B21079
:1001200032141230B100051D9A28331483160113BE
:10013000831208003310831601178312080032114E
:100140000130B7008B132030370783169B001C1437
:100150001A088312A400A500C030A5061030370786
:1001600083169B001C141A088312A3000030370763
:1001700083169B001C141A088312A2008B17331CD1
:10018000C72822090339A200A309A409A509220846
:100190002D02031D122923082E02031D12292408F3
:1001A0002F02031D122901303702031DDC283E18DF
:1001B000DC283E143F14B92102303702031DE52824
:1001C000BE18E528BE143F14BB2103303702031DBF
:1001D000EE283E19EE283E153F14BD2104303702AB
:1001E000031DF728BE19F728BE153F14BF2105309F
:1001F0003702031D00293E1A00293E163F14C12173
:1002000006303702031D0929BE1A0929BE163F14FC
:10021000C32107303702031D12293E1B12293E1746
:100220003F14C521B70A0830370203180800A22876
:100230000130B600B400B500B70085018701B213E4
:10024000E9218920B40B3129031085190314BA0D53
:10025000F0303A0203195829B50B31299630B50010
:100260006421321D21293211331C3B292D09033908
:10027000AD00AE09AF092F1CB2132F1C2129B21BF0
:1002800021292E182129B2178B1320303707BC00E3
:100290002F08BB008A2110303707BC002E08BB0096
:1002A0008A2100303707BC002D08BB008A218B173C
:1002B00085018701B70AB6010130B5000830370261
:1002C000031C2129EC210800013037020319D02139
:1002D000023037020319D521033037020319D82120
:1002E000043037020319DB21053037020319E021FE
:1002F000063037020319E321073037020319E621DC
:1003000008003F1C08003F101030BC003E08BB0036
:100310008A2108008B133B0883161C159A00831250
:100320003C0883169B0055309D00AA309D009C140C
:1003300064009C1898291C1183128B1708008316DF
:1003400000309B001C141A088312BD008316103065
:100350009B001C141A088312BE00FF30D000D41575
:10036000D515D615D715D815D915DA15DB15DC1521
:100370000800F130C829F230C829F430C829F83013
:10038000C8291F30CC292F30CC294F30CC29080068
:10039000BE050F30D2040800BE05F030D2040800BC
:1003A00010308506023087060800203085060800D8
:1003B00021308506080002308506023087060800D5
:1003C00018308706080021308706080009308706A4
:1003D00008003E18D02108003E08D200031D080086
:1003E0001130BE00D2000800B601B401B5013D1CB9
:1003F000FC29BD01BD14FE29BD013D143D08B60018
:100400006400022A032A042A052A062AB51B0516B7
:10041000B51F0512B40B002AB50B002A0310B60C49
:10042000B608031D002A0030BC003D08BB008A212D
:1004300008008F08031908008F01D00F542BD00A31
:100440000E305205031D332A541D292AD401541697
:10045000412AD41D2E2AD4015416412A541E412A61
:10046000D401D414412AD41C382AD4015415412A69
:10047000541D3D2AD401D415412A541E412AD401C9
:10048000541509305205031D542A551D4A2AD50119
:100490005516622AD51D4F2AD5015516622A551EBA
:1004A000622AD501D514622AD51C592AD5015515C1
:1004B000622A551D5E2AD501D515622A551E622A6B
:1004C000D50155150B305205031D752A561D6B2A93
:1004D000D6015616832AD61D702AD6015616832AAF
:1004E000561E832AD601D614832AD61C7A2AD60110
:1004F0005615832A561D7F2AD601D615832A561EE5
:10050000832AD601561507305205031D962A571D1A
:100510008C2AD7015716A42AD71D912AD70157161E
:10052000A42A571EA42AD701D714A42AD71C9B2A71
:10053000D7015715A42A571DA02AD701D715A42AD9
:10054000571EA42AD701571506305205031DB72A96
:10055000581DAD2AD8015816C52AD81DB22AD8016F
:100560005816C52A581EC52AD801D814C52AD81C21
:10057000BC2AD8015815C52A581DC12AD801D8153A
:10058000C52A581EC52AD80158151030BD18193073
:100590005205031DDA2A591DD02AD9015916E82A15
:1005A000D91DD52AD9015916E82A591EE82AD90198
:1005B000D914E82AD91CDF2AD9015915E82A591D6E
:1005C000E42AD901D915E82A591EE82AD901591572
:1005D0005030BD1859305205031DFD2A5A1DF32A0B
:1005E000DA015A160B2BDA1DF82ADA015A160B2BF0
:1005F0005A1E0B2BDA01DA140B2BDA1C022BDA0150
:100600005A150B2B5A1D072BDA01DA150B2B5A1E24
:100610000B2BDA015A156030BD1869305205031DE5
:10062000202B5B1D162BDB015B162E2BDB1D1B2BE2
:10063000DB015B162E2B5B1E2E2BDB01DB142E2B1E
:10064000DB1C252BDB015B152E2B5B1D2A2BDB0115
:10065000DB152E2B5B1E2E2BDB015B152030BD180E
:1006600029305205031D432B5C1D392BDC015C1620
:10067000512BDC1D3E2BDC015C16512B5C1E512BDB
:10068000DC01DC14512BDC1C482BDC015C15512BEC
:100690005C1D4D2BDC01DC15512B5C1E512BDC014C
:1006A0005C1581213E08D2005008D1000C30540561
:1006B000031D05120C305505031D85120C3056051F
:1006C000031D05100C305705031D85100C3058050F
:1006D000031D87100C305905031D07100C305A05F7
:1006E000031D87120C305B05031D07120C305C05DF
:1006F000031D871151080E020318A62B1230540552
:10070000031D051612305505031D851612305605BA
:10071000031D051412305705031D851412305805AA
:10072000031D871412305905031D071412305A0592
:10073000031D871612305B05031D071612305C057A
:10074000031D8715FF305002031908008F08031D91
:100750000800892051080E02031CA62B18305405EE
:10076000031D051206305405031D051618305505E6
:10077000031D851206305505031D851618305605D4
:10078000031D051006305605031D051418305705C6
:10079000031D851006305705031D851418305805B4
:1007A000031D871006305805031D8714183059059E
:1007B000031D071006305905031D071418305A058C
:1007C000031D871206305A05031D871618305B0576
:1007D000031D071206305B05031D071618305C0564
:0E07E000031D871106305C05031D87150800F8
:084000000A00030007000100A3
:02400E00CC33B1
:10420000010003000300030003000200020002009B
:1042100002000000000000000000FF00FF00FF009F
:10422000000000000000000000000000000000008E
:104230000000C000C000C000C000FF00FF00FF0081
:104240000100C300F300CF00FF00C300F300CF0064
:10425000FF00C300F300CF00FF00FF00FF00FF00DE
:10426000FF00FF00FF00FF00FF00FF00FF00FF0056
:10427000FF00FF00FF00FF00FF00FF00FF00FF0046
:10428000FF00FF00FF00FF00FF00FF00FF00FF0036
:10429000FF00FF00FF00FF00FF00FF00FF00FF0026
:1042A000FF00FF00FF00FF00FF00FF00FF00FF0016
:1042B000FF00FF00FF00FF00FF00FF00FF00FF0006
:1042C000FF00FF00FF00FF00FF00FF00FF00FF00F6
:1042D000FF00FF00FF00FF00FF00FF00FF00FF00E6
:1042E000FF00FF00FF00FF00FF00FF00FF00FF00D6
:1042F000FF00FF00FF00FF00FF00FF00FF00AA001B
:00000001FF
